:020000040000FA
:040000000000D22802
:08000800FE000308FF00830164
:100010000C11C90803190D28C903F723B90B44288B
:100020001E30B900331F1728E90B17283313BB0BF9
:1000300044280530BB00301D1F2830112028301502
:10004000BA0B44280230BA009127051F2C28B31C94
:100050002B28B3102C28B314DF0803193A28DF0B20
:100060003A285F243311B10133124308E000B31280
:10007000B2103215BD0B44283C30BD00E008031916
:100080004328E00B4428B3167F088300FE0E7E0E43
:10009000090082077E340C34B6349E34CC34DA3412
:1000A000FA340E34FE34DE340034803482070034F7
:1000B0000134013402340334033404340434053489
:1000C000063406340734083408340934093400345B
:1000D00082070C347234EC348034B634CC34DE34E1
:1000E0007E3480340C340C3472340C34F234A0344A
:1000F000A034B834A0340034BC34EE34F034B0341E
:10010000E9341034FE3480347E34DA34FA34803406
:100110009E340E34CC3480347E34CC3480347E34FF
:10012000DA340A34EE347034EE34A1340034BC34A2
:10013000EE34F034EE340434B834E234E2340334D0
:10014000B834A83405347234B8347034BC3406344E
:10015000EC34B834F03470343C340434DC3472346D
:10016000F0340434F0343834B0340434CE34083449
:10017000B0340434BC34B834F03404347C3438340F
:10018000F0340434F034F23470340434A034F234F3
:10019000CE340934A834B8340034A8348834B834A0
:1001A000BC34F234053084008001840A7B300402C0
:1001B000031DD428640007309F00831603130F30FB
:1001C00081008601103085008312031385018601AA
:1001D00083120313313090000B30970001309600EA
:1001E000A030950037247830C5000230B900BA003D
:1001F000BB00BC00BD00B21032154308E000B312D2
:10020000C0308B00831603130C158312031383165F
:1002100003130E30860083120313861D9029831664
:100220000313860183120313003095234430952372
:10023000CE233F08CB004008CC00B414B425E02402
:10024000A72477233E1827293630952329293230D1
:1002500095237723CE233508CB003608CC00B41481
:10026000B425E024E023C02464003508CB00360820
:10027000CC00B414B42506257830C9008E233E1C6A
:100280004429051385134B295E21CB21301B4B29B3
:10029000301A4B29A9210322331D3429B3195329BC
:1002A0007830C5005729450303195729C503450868
:1002B000C9008E230322A92164004C294008D900DB
:1002C0003F08D800E230DC000430DB006325DE1894
:1002D00090294008D9003F08D800DA30DC00FD3012
:1002E000DB0063255E1990294108D900D801FA3056
:1002F000DC00DB016325DE1890294208D900D80113
:10030000FA30DC00DB016325DE1890294308D900B0
:10031000D8016430DC00DB016325DE189029080079
:10032000831603138601831203130930BE00BF0135
:10033000FA30C0000A30C1000030C2001E30C300D5
:100340005F24051385174611C610461028309523E3
:10035000A129DB013608D9003508D800410840073B
:10036000DC000318DB0A3F08DB076325DE19C92917
:10037000DB013608D9003508D8003F08DB0041080A
:100380004002DC00031CDB0363255E1ECA2905173F
:10039000CA2905130800B31E0800C2080319080083
:1003A0003508D8003608D9003F08DB004008DC00DB
:1003B0004108DC07031CDD29DB0A4208DC07031CBB
:1003C000E229DB0A63255E1DFA293508D8003608C4
:1003D000D9003F08DB004008DC004108DC020318BC
:1003E000F229DB034208DC020318F729DB0363254B
:1003F000DE18080005138517603095230322B31E0D
:100400000800FA290800831603130E3086008312B1
:100410000313B3110619142A331E102A3312112A9A
:100420003316B3152C22262A86181B2A331A212AA2
:10043000B2143211212A8619262A331A212A32159A
:10044000B210331E252ACE22262A2C22831603130D
:100450008601831203130800B3128513B3158316A4
:1004600003138601831203134610C6104611331579
:100470000730DF00331E492A3118B42AB118A22AE6
:100480003119912AB119802A311A702AB11A612AB8
:10049000B42AB218562A3118A22AB118912A311951
:1004A000802AB119702A311A612AB42A3118612AB6
:1004B000B11A702A311A802AB119912A3119A22A47
:1004C000B42A2030B100331A6B2A583032199523E0
:1004D000B218B123CC2A1830952358309523CC2A52
:1004E0001030B100331A7A2A543032199523B218D9
:1004F000B123CC2A4308CC00CB01B425D924CC2A83
:100500000830B100331A8A2A503032199523B218B4
:10051000B123CC2A4208CC00CB01B414B425062563
:10052000CC2A0430B100331A9B2A4C30321995235F
:10053000B218B123CC2A4108CC00CB01B414B425A5
:100540000625CC2A0230B100331AAC2A48303219C1
:100550009523B218B123CC2A3F08CB004008CC0029
:10056000B414B4250625CC2A0130B100331ABE2AB2
:100570005C3032199523B218B123CC2A3E18C62A12
:10058000A001B830A100A830A200CC2AB830A00049
:10059000E230A100E230A20032100800B3150730AB
:1005A000DF00B118DC2A3119282BB1193B2B311A85
:1005B0004E2B3118612B08008619FF2A0430D80011
:1005C000E230D9003230D9020318E72AD8034108B3
:1005D000D9020318EC2AD8033F08DB004008DC00EE
:1005E0006325DE1CFF2A4619FA2A0130C0070318CA
:1005F000BF0A222B0A30C0070318BF0A222B861815
:10060000222BD8013230D900DA30D907031C092B4C
:10061000D80A4108D907031C0E2BD80AFD30D80789
:100620003F08DB004008DC0063255E1D222B4619D5
:100630001E2B0130C002031CBF03222B0A30C00254
:10064000031CBF0383160313860183120313AC2A12
:1006500086192F2BFA304102031DC10A352B86184B
:10066000352B00304102031DC1038316031386019D
:10067000831203139B2A8619422BFA304202031D70
:10068000C20A482B8618482B00304202031DC203C1
:10069000831603138601831203138A2A8619552BA6
:1006A00064304302031DC30A5B2B86185B2B0A30A0
:1006B0004302031DC303831603138601831203132E
:1006C0007A2A8618642B3E148619672B3E108316EF
:1006D0000313860183120313BE2A64002D08AE00A3
:1006E0002D08AF00AF0B722BAE0B702B080030192A
:1006F000772B4714C7144715FF30C9008E23FF30EE
:10070000C9008E23FF30C9008E233019852B471076
:10071000C7104711FF30C9008E2308006400C908C4
:10072000031D8E2B3C30C9000800A7004610C610E0
:100730004611CE232708B8006820B700B80AB70BC7
:10074000A22B080064002108A0002208A10038089C
:100750006820A2006400C908031DAA2B3C30C90010
:100760009E2BA7004610C6104611E0232708B800AC
:100770006820B700B807B803B70BBF2B08006400A8
:100780002108A2002008A10038086820A000640009
:10079000C908031DC72B3C30C900BB2B0430B8006F
:1007A000B80BD32B080064002108A0002208A10088
:1007B000A2016400C908031DD92B3C30C900D02B0D
:1007C0000430B800B80BE52B080064002108A20033
:1007D0002008A100A0016400C908031DEB2B3C30D8
:1007E000C900E22B64003C30C9008E230800461883
:1007F0002014C618211446192214481C112C051562
:1008000020088600471C092C301D092C0130860564
:10081000092C461E0D2C301D06100510C801C814E9
:100820000800C81C252C051421088600C71C1D2C97
:10083000301D1D2C013086051D2CC61E212C301D9F
:1008400006108510C8014815080085142208860086
:10085000471D2F2C301D2F2C013086052F2C461FB5
:10086000332C301D06100511C8014814080007304C
:10087000EA003E308400AB0143248000840AAB0AC6
:10088000EA0B3C2C080055242C08A600AB0A552482
:100890002C082602031D4E2C2C080800031C522C89
:1008A0002C08532C2608B01508002B0883160313B8
:1008B0009B001C141A0883120313AC0008000B08D9
:1008C000AA008B13073083120313EA008312031369
:1008D0003E308400AB018312031300087A24840A9B
:1008E000AB0A83120313EA0B6B2C831203132A083F
:1008F0008B000800AC00A7008224AB0A2708AC00DC
:1009000082240800831603139C18842C1C15831260
:1009100003132B08831603139B00831203132C0865
:10092000831603139A008316031355309D00AA30D3
:100930009D009C149C189A2C8312031308008316A4
:1009400003139C18A12C1C11831203130800210807
:10095000A0002208A1002308A200F22364002108BD
:10096000A0002208A1002408A200F22364002108AC
:10097000A0002208A1002508A200F22364000800BC
:100980002108A2002008A1002508A000F22364008D
:100990002108A2002008A1002408A000F22364007E
:1009A0002108A2002008A1002308A000F22364006F
:1009B00008005008A2005108A1005208A000080039
:1009C0004B08D8004C08D9000330DB00E830DC00CD
:1009D00063255E1DFE2C4B08D8004C08D900FF3063
:1009E000DB009C30DC006325DE1CFE2C5008A500DB
:1009F0005108A40024145208A30008005108A500BF
:100A000025145208A4005308A30008003012301B1C
:100A10005D2D4B08D8004C08D9000430DB00E230D3
:100A2000DC006325DE1C192D3E309523CE233016C5
:100A300008004B08D8004C08D900FD30DB00DA3044
:100A4000DC0063255E1D292D39309523CE23301619
:100A500008004B08D8004C08D9000330DB00E83010
:100A6000DC0063255E1D4E2D4B08D8004C08D900D4
:100A7000FF30DB009C30DC006325DE1C4E2D051FA3
:100A8000432DC616442DC61246134611C6145008EF
:100A9000A2005108A1005208A0000800051F522D15
:100AA0004617532D4613C6124615C6105108A2000C
:100AB0005208A1005308A0000800051385170C3048
:100AC0009523CE230800DE01DD01341C6C2DD71BDD
:100AD0005D14DA1BDD14702DD81B5D14DB1BDD14D7
:100AE000DD080319812D01305D02031D7A2D5E158D
:100AF0005E16080002305D02031D812DDE14DE1536
:100B00000800341C932D341057085A02031D892DF8
:100B1000932D57085A020318902DDE14DE15080095
:100B20005E155E16080058085B02031D982DA22D65
:100B300058085B0203189F2DDE14DE1508005E15B1
:100B40005E16080059085C02031DAA2D5E145E168D
:100B5000DE15080059085C020318B12DDE14DE15FD
:100B600008005E155E1608004A08CD004B08CE004E
:100B70004C08CF00D601D501D401D301D201D10157
:100B8000D001B0133418C82DCA01CB1FD62DCB2DE0
:100B9000CA1FD62DCA09B017CC09CB090130CC0722
:100BA000031CD62DCB07031CD62DCA0A34104C1CAF
:100BB000DB2D01300927CC1CDF2D023009274C1D0D
:100BC000E32D04300927CC1DE72D083009274C1EE2
:100BD000ED2D0630092701301227CC1EF32D0230EF
:100BE0000927033012274C1FF92D0430092706303E
:100BF0001227CC1F012E083009270230122701309E
:100C00001B274B1C092E06300927053012270230FE
:100C10001B27CB1C112E023009270130122705306B
:100C20001B274B1D192E04300927023012270130D3
:100C30002427CB1D212E083009270430122702302B
:100C400024274B1E292E063009270930122704308D
:100C50002427CB1E332E02300927093012270130FA
:100C60001B27083024274B1F3F2E0430092708304C
:100C7000122703301B270630242701302D27CB1FD6
:100C80004B2E083009270630122707301B27023069
:100C9000242703302D274A1C572E063009270330FE
:100CA000122705301B270530242706302D27CA1CA4
:100CB000632E023009270730122701302427033022
:100CC0002D27013036274A1D712E043009270430A4
:100CD000122701301B270230242706302D2702302F
:100CE0003627CA1D7F2E0830092708301227023008
:100CF0001B270430242702302D27053036274A1EB3
:100D00008D2E063009270730122705301B270830A3
:100D1000242704302D2701303F27CA1E9B2E023086
:100D200009270530122701301B27073024270930F7
:100D30002D2702303F274A1FA92E043009270330F0
:100D40001B270430242709302D2701303627043093
:100D50003F270A30D608031DC62ED600D508031D2E
:100D6000C62ED500D408031DC62ED400D308031DFB
:100D7000C62ED300D208031DC62ED200D108031DF3
:100D8000C62EB41CC52EB410C62ED100B01FED2E39
:100D90000A305102031DCF2E0B30D100ED2E0A3048
:100DA0005202031DD62E0B30D200ED2E0A30530214
:100DB000031DDD2E0B30D300ED2E0A305402031D2F
:100DC000E42E0B30D400ED2E0A305502031DEB2E1D
:100DD0000B30D500ED2E0B30D60056084920D6003A
:100DE00055084920D50054084920D400530849200B
:100DF000D30052084920D20051084920D1005008A0
:100E00004920D0004D08CA004E08CB004F08CC0046
:100E10000800D0070A30500203180F2F08000A30CC
:100E2000D0020130D1070A3051020318182F0800F0
:100E30000A30D1020130D2070A3052020318212FA2
:100E400008000A30D2020130D3070A3053020318D7
:100E50002A2F08000A30D3020130D4070A30540286
:100E60000318332F08000A30D4020130D5070A30A6
:100E7000550203183C2F08000A30D5020130D6076E
:100E80000A30560208006527A030E400E40B462F24
:100E90005A27E4016400E40B4F2F3017080085192E
:100EA0004A2FE4016400E40B562F4D2F851D522F6D
:100EB0003013080085150130E400E40B5D2F831624
:100EC000031385158312031300348316031385114E
:100ED0008312031385110130E400E40B6D2F0034FD
:100EE0001430E400E40B722F00340830E50065276D
:100EF0005A27851D031085190314E10C7027E50B93
:100F0000772F0034E1000830E5006527E10C031C71
:100F10008B2F5A278C2F652770275A27E50B852F93
:100F200000346400B31BA02F4327301B0800CC30D3
:100F3000822744308227B3170230E90033170800B4
:100F4000331B08004327301B0800CC308227BE30FB
:100F5000822775276108E30075276108E200B31353
:100F60003411E21FB42F34150F306305341DBC2F2C
:100F7000E400E40364090F395620E600E20EF03085
:100F8000E205F030E305630E6204E700341DCA2F6A
:100F9000E709E70A341DD02FE6080319D02FE7032D
:100FA0006708E400E8010310E70DE80DE70DE80D20
:100FB000E70DE80D6408E7070318E80A6408E70787
:100FC0000318E80A6608E7070318E80A6708E60056
:100FD0006808E700E801341DF22FE609E60A031964
:100FE000E703E7096608B6006708B50008000028AF
:100FF00000280028002800280028002800280028B1
:02400E00341E5E
:1042000000000000010001002C002C000A000A0040
:08421000000000001E001E006A
:00000001FF
